:100000000C9434000C943E000C943E000C943E0082
:100010000C943E000C943E000C943E000C943E0068
:100020000C943E000C943E000C943E000C943E0058
:100030000C943E000C943E000C943E000C943E0048
:100040000C943E000C943E000C943E000C943E0038
:100050000C943E000C943E000C943E000C943E0028
:100060000C943E000C943E0011241FBECFEFD8E04C
:10007000DEBFCDBF0E9446000C9467000C940000C8
:1000800002C0000001970097E1F7089514B880EDD1
:100090008AB92FEF80E09DE7000001970097E1F714
:1000A0002BB980E197E2000001970097E1F71BB8B8
:1000B00080E197E2000001970097E1F72BB980E11A
:1000C00097E2000001970097E1F71BB8E3CFF8949F
:0200D000FFCF60
:00000001FF
